:020000021000EC
:10F800000C9446FC0C9466FC0C9466FC0C9466FC10
:10F810000C9466FC0C9466FC0C9466FC0C9466FCE0
:10F820000C9466FC0C9466FC0C9466FC0C9466FCD0
:10F830000C9466FC0C9466FC0C9466FC0C9466FCC0
:10F840000C9466FC0C9466FC0C9466FC0C9466FCB0
:10F850000C9466FC0C9466FC0C9466FC0C9466FCA0
:10F860000C9466FC0C9466FC0C9466FC0C9466FC90
:10F870000C9466FC0C9466FC0C9466FC0C9466FC80
:10F880000C9466FC0C9466FC0C9466FC11241FBE60
:10F89000CFEFD0E4DEBFCDBF11E0A0E0B1E0E0ECFF
:10F8A000FFEF01E00BBF02C007900D92A030B1073F
:10F8B000D9F71BBE12E0A0E0B1E001C01D92A93053
:10F8C000B107E1F70E94B7FD0C94DEFF0C9400FC39
:10F8D000982F8091C00085FFFCCF9093C6000895BB
:10F8E0001F93982F82958F708A3080F0282F295A85
:10F8F000892F8F708A3080F4182F105D822F0E941C
:10F9000068FC812F0E9468FC1F910895282F205DBC
:10F91000892F8F708A3080F3182F195A822F0E94F6
:10F9200068FC812F0E9468FC1F910895EF92FF925E
:10F930000F931F932898EE24FF2487018091C00025
:10F9400087FD17C00894E11CF11C011D111D81E009
:10F95000E81689E0F8068DE3080780E0180770F3E1
:10F96000E0910101F091020109958091C00087FFAB
:10F97000E9CF289A8091C6001F910F91FF90EF90D8
:10F9800008950F931F930E9496FC182F0E9468FC05
:10F990000E9496FC082F0E9468FC113668F01755EB
:10F9A000013678F4003308F000531295107F802F51
:10F9B000810F1F910F910895103390F3105301366A
:10F9C00088F307551295107F802F810F1F910F919B
:10F9D0000895282F882351F090E08091C00087FF80
:10F9E000FCCF8091C6009F5F9217B8F308951F93D4
:10F9F000182F0E9496FC803281F0809100018F5F69
:10FA000080930001853011F01F910895E09101016C
:10FA1000F091020109951F91089584E10E9468FC0C
:10FA2000812F0E9468FC80E10E9468FC1F9108956C
:10FA30000E9496FC803271F0809100018F5F80936C
:10FA40000001853009F00895E0910101F091020173
:10FA50000995089584E10E9468FC80E10E9468FC99
:10FA60000895DF93CF9300D000D0CDB7DEB78823C1
:10FA700009F076C041E050E020E030E0289A198299
:10FA80001A821B821C8289819A81AB81BC81805839
:10FA90009E43A040B040A0F489819A81AB81BC8193
:10FAA0000196A11DB11D89839A83AB83BC83898193
:10FAB0009A81AB81BC8180589E43A040B04060F3E6
:10FAC000289819821A821B821C8289819A81AB81B3
:10FAD000BC8180509A4FA040B040A0F489819A81A7
:10FAE000AB81BC810196A11DB11D89839A83AB8333
:10FAF000BC8389819A81AB81BC8180509A4FA040A0
:10FB0000B04060F32F5F3F4F241735070CF4B6CF9A
:10FB100019821A821B821C8289819A81AB81BC81E5
:10FB200080509147A240B040A0F489819A81AB8176
:10FB3000BC810196A11DB11D89839A83AB83BC83CF
:10FB400089819A81AB81BC8180509147A240B040AD
:10FB500060F30F900F900F900F90CF91DF91089569
:10FB6000482F50E04115510509F086CFD1CFEF92D3
:10FB7000FF920F931F93CF93DF93000094B714BEAF
:10FB8000809160008861809360001092600091FF16
:10FB9000A0C189E18093C4001092C50088E18093E0
:10FBA000C10086E08093C2005098589A209A83E062
:10FBB0000E9431FD81E00E9431FD0E9496FC80335D
:10FBC000B9F18133C1F1803409F455C0813409F4AD
:10FBD0005BC0823409F46AC0853409F46DC0803595
:10FBE00039F1813509F444C1823511F1853509F4C3
:10FBF00069C0863509F471C0843609F4CEC08437F3
:10FC000009F472C0853709F449C1863709F44AC03E
:10FC1000809100018F5F80930001853071F6E09143
:10FC20000101F091020109950E9496FC803349F68A
:10FC30000E9418FDC2CF0E9496FC803249F784E1F1
:10FC40000E9468FC81E40E9468FC86E50E9468FCD2
:10FC500082E50E9468FC80E20E9468FC89E40E94C0
:10FC600068FC83E50E9468FC80E50E9468FC80E1F6
:10FC70000E9468FCA2CF0E9496FC8638C8F20E94BF
:10FC800096FC0E9418FD99CF0E9496FC803809F4DA
:10FC900001C1813809F4FAC0823809F4F3C0883907
:10FCA00009F4ECC080E00E94F7FC87CF84E10E9459
:10FCB000E9FC0E9418FD81CF85E00E94E9FC0E94CA
:10FCC00018FD7BCF0E9496FC809303010E9496FC56
:10FCD000809304010E9418FD70CF84E00E94E9FC2B
:10FCE00080E00E94F7FC69CF0E9496FC8093060298
:10FCF0000E9496FC809305020E9496FC853409F4CC
:10FD0000E2C0809108028E7F8093080280910301F7
:10FD100090910401880F991F90930401809303012F
:10FD20000E9496FC803209F048CF84E10E9468FC72
:10FD30008091050290910602009709F4C0C000E08E
:10FD400010E0E0910301F09104010DC021FF2AC1F0
:10FD50003196F0930401E09303010F5F1F4F0817E2
:10FD6000190708F0ACC02091080220FFEFCFF999E5
:10FD7000FECFF2BDE1BDF89A80B50E9468FCE0912B
:10FD80000301F09104013196F0930401E093030123
:10FD90008091050290910602E0CF0E9496FC80932C
:10FDA00006020E9496FC80930502809108028E7FD5
:10FDB000809308020E9496FC853429F48091080201
:10FDC00081608093080245E0E42E41E0F42EF701C3
:10FDD000119281E0E538F807D9F7809105029091FA
:10FDE0000602892B89F000E010E00E9496FCF801E1
:10FDF000EB5FFE4F80830F5F1F4F80910502909154
:10FE000006020817190788F30E9496FC803209F051
:10FE1000FFCE8091080280FF62C060910502709160
:10FE2000060261157105E9F040910301509104014A
:10FE30009A01FB01EB5FFE4FF999FECF32BD21BD68
:10FE4000D7018D917D0180BDFA9AF99A2F5F3F4FBE
:10FE5000AE17BF0789F7460F571F50930401409311
:10FE6000030184E10E9468FC80E10E9468FCA5CE49
:10FE70000E9418FD88E080936000FFCF83E00E941D
:10FE8000F7FC9BCE80E10E94F7FC97CE81E00E94B8
:10FE9000F7FC93CE82E00E94F7FC8FCE0E9496FC86
:10FEA000803209F0B5CE84E10E9468FC8EE10E94A8
:10FEB00068FC87E90E9468FC85E00E9468FC80E19C
:10FEC0000E9468FC7ACE80910802816080930802CB
:10FED00027CFE0910101F091020109955ACE80915E
:10FEE000030190910401880F991F9093040180935E
:10FEF00003018091050280FF09C080910502909165
:10FF0000060201969093060280930502F999FECFAE
:10FF10001127E0910301F0910401C5E0D1E0809147
:10FF2000050290910602103091F400915700017083
:10FF30000130D9F303E000935700E8950091570092
:10FF400001700130D9F301E100935700E895099061
:10FF500019900091570001700130D9F301E000932E
:10FF60005700E8951395103898F011270091570025
:10FF700001700130D9F305E000935700E895009136
:10FF8000570001700130D9F301E100935700E89563
:10FF90003296029709F0C7CF103011F00296E5CFE4
:10FFA00011245FCF84910E9468FC8091050290919A
:10FFB0000602E0910301F0910401CACEF894FFCF4C
:040000031000F800F1
:00000001FF
